:10000000ABC00000C5C00000C3C00000C1C00000FC
:10001000BFC00000BDC00000BBC00000B9C00000F0
:10002000B7C00000B5C00000B3C00000DFC60000CC
:10003000AFC00000ADC00000ABC00000A9C0000010
:10004000A7C00000A5C00000A3C00000A1C0000020
:100050009FC000009DC000009BC0000099C0000030
:1000600097C0000095C0000093C0000091C0000040
:100070008FC000001C0350004900550020004800BC
:10008000490044002000560031002E0030003000AE
:1000900000000C0350004900550049004F000000CB
:1000A000120341004E00440041004D00490052003F
:1000B0004F0000000C034E00540044004500430074
:1000C00000000403090409022900010100C03209EB
:1000D0000400000203000000092111010001222098
:1000E0000007058103100001070502031000010647
:1000F00000FF0901A1010902150025FF75089510EF
:1001000081020903150025FF750895109102C009A9
:10011000021200010100C0320904000000000000CA
:100120000012011001000000082F0D401001000115
:1001300002000112011001000000082F0D20100123
:10014000000102000112010001FF00000847050242
:10015000100001010200010011241FBECFEFD2E008
:10016000DEBFCDBF11E0A0E0B1E0E6E2F2E102C007
:1001700005900D92AA33B107D9F721E0AAE3B1E0C7
:1001800001C01D92A537B207E1F726D00C941109E2
:1001900037CF4AB121E030E0B90102C0660F771FC6
:1001A0008A95E2F7CB01462B4AB99BB1809589230A
:1001B0008BB908954AB121E030E0B90102C0660F61
:1001C000771F8A95E2F7CB01962F909594239AB9E1
:1001D0009BB1892B8BB90895CF93DF9300D0CDB716
:1001E000DEB7109245011092440120D389E190E0DE
:1001F0009093CD008093CC0086E08093CA0010924B
:10020000C80088E18093C900539A5A9A7894A8E468
:10021000B1E0E0E5F1E089E09FEF815009F08AC0AC
:1002200088E080933A0106E588D2E0D780914401C6
:1002300090914501893E934014F084E0AADF8091BB
:10024000440190914501813D974034F084E0B2DF54
:1002500010924501109244018091500180933B011E
:100260008091520180933C01809153019091510102
:1002700092FF63C0806880933D018091C80085FF34
:10028000FCCF0093CE00F12CE12C8091C80087FFB9
:1002900056C08091C80087FD5CC0198110933E0153
:1002A000FA80F0923F0185E01F3F21F42FEFF21614
:1002B00009F49CC06EDF9091490180914B0115FDBE
:1002C00097C09F77909349018F7780934B019091CE
:1002D000490180914B0116FD90C09F7B909349018D
:1002E0008F7B80934B019091490180914B01F5FCEC
:1002F00089C09D7F909349018D7F80934B01212F71
:10030000206E20933E018091490117FD80C08B7FB4
:10031000809349019F2D906A90933F0180914B01FA
:10032000F7FC77C08B7F80934B012093480190931B
:100330004A017ACF9D93119270CF8F779CCF8FEF28
:10034000E81AF80A90E1E91697E2F90609F09DCF5C
:100350006BCF8091C80087FF12C08091CE008E3A8B
:1003600009F03FC010923A01E0913A01E33050F0B9
:1003700010923A0180913A018230E8F08ACF8FEFF3
:100380009FEFEDCFF0E0E55CFE4F80819091C800DB
:1003900095FFFCCF8093CE0080913A018F5F8093D0
:1003A0003A01E2CF2FEFE21AF20A90E1E91697E262
:1003B000F9060CF039CF9091C80097FFF3CF9091D8
:1003C000C8002FEF3FEF97FD2091CE00E1E0F0E075
:1003D000EC0FFD1FE80FF11D20838F5F80933A0122
:1003E000C9CF8F3D09F055CF59D253CFE3DE63CF4C
:1003F000906890934901806868CF90649093490118
:1004000080646FCF926090934901826076CF846060
:100410007FCF846088CF292F332723303105F1F136
:1004200058F421303105D1F02230310529F190E026
:1004300080E0F0E0E0E00EC089E090E0E8EDF0E080
:100440002132310539F080E290E0EFEEF0E0223227
:10045000310569F7DA01ED93FC930895E0914001CD
:10046000F0914101EE0FFF1FEE5EFE4F0190F08113
:10047000E02D82E190E0EECF80914001909141012A
:10048000880F991FFC01E45FFE4F0190F081E02D81
:10049000875D9E4FDC018D919C91DCCF9927813047
:1004A000910589F058F0029711F6E0914001F09122
:1004B0004101EE0FFF1FE050FF4F0DC0E2ECF0E0F6
:1004C000849190E0C7CFE0914001F0914101EE0F9F
:1004D000FF1FEA5FFE4F0190F081E02DF1CF0895FC
:1004E00008958091400190914101892B41F061E094
:1004F00084E391E0A9D361E08FE291E0A5D38091FC
:10050000E20084608093E200089580916E018E3A4B
:1005100041F58091400190914101892B11F5809125
:1005200044019091450101969093450180934401C7
:1005300080916D011092E90087FD14C08091E80060
:1005400080FFFCCF8091E800877F8093E80068E01F
:1005500070E080E591E0B0D28091E8008E778093E2
:10056000E80008958091E800877F8093E80068E0C4
:1005700070E088E491E044D28091E8008B77EFCF7F
:10058000CF93DF93CDB7DEB760970FB6F894DEBF99
:100590000FBECDBF80916E01833009F458C070F456
:1005A000813089F1823009F49AC060960FB6F894D0
:1005B000DEBF0FBECDBFDF91CF9108958A3009F421
:1005C00073C08B3009F45CC0893079F780916D017C
:1005D000813259F78091E800877F8093E80060E1DD
:1005E00070E0CE01019668D28091E8008E7780930A
:1005F000E80080E1FE013196A8E5B1E001900D929E
:100600008A95E1F7D2CF80916D01813A71F6909190
:100610006F0180E1E9E1F1E0DE01119601900D92B8
:100620008A95E1F71092E9008091E800877F809336
:10063000E80091119093F10060E170E0CE01019625
:10064000DFD18091E8008B778093E800AECF809176
:100650006D01813A09F0A9CF8091E800877F8093EE
:10066000E8008091E80080FFFCCF80911801809322
:10067000F1008091E8008E778093E80021D395CF38
:1006800080916D01813209F090CF8091E800877FE1
:100690008093E80015D390916F0181E0911101C022
:1006A00080E08093180181CF80916D01813209F043
:1006B0007CCF8091E800877F8093E80001D3809110
:1006C0006F019091700136E0969587953A95E1F724
:1006D0008C7F9370909343018093420166CF809109
:1006E0006D01813A09F061CF8091E800877F8093A6
:1006F000E8008091E80080FFFCCF8091420190915A
:1007000043019695879596958795B1CF8091E8009E
:1007100083FF11C08091710190917201892B59F46E
:100720008091400190914101009709F4EECE01972C
:10073000029708F425CF0895089580914001909183
:100740004101892B09F46AC0809148018093190105
:1007500080931A0180931B0180931C0180914A01B0
:1007600080931D0180931E0180931F0180932001BF
:10077000809149018093210180914B018093220156
:100780008FEF80932301809324018093270180932E
:10079000280181E08093E9008091E80080FF15C086
:1007A0008091440190914501019690934501809379
:1007B000440150E040E060E170E089E191E084D0E4
:1007C0008091E8008E778093E80082E08093E900D2
:1007D0008091E80082FF19C08091E80085FF10C079
:1007E0008091440190914501019690934501809339
:1007F000440150E040E060E170E088E591E0B2D073
:100800008091E8008B778093E80088E0E8E5F1E0EC
:10081000A0E5B1E001900D928A95E1F70895F9996C
:10082000FECF92BD81BDF89A80B50895A89584B792
:10083000877F84BF0FB6F894A89580916000886187
:1008400080936000109260000FBE80E890E00FB6C9
:10085000F89480936100909361000FBE90E080E077
:10086000DEDF833070F490E090934101809340018B
:1008700080914001909141019093470180934601FE
:10088000A6C21092410110924001F2CFF999FECF19
:1008900092BD81BD60BDFA9AF99A08958091460192
:1008A000909147010196833091054CF49093470154
:1008B000809346016091460190E080E0E7CF10927E
:1008C000470110924601F6CFAF92BF92CF92DF92CE
:1008D000FF920F931F93CF93DF936C01EB018A017B
:1008E0000ED2F82E811124C00115110539F0F8013E
:1008F00080819181C81BD90BC80ED91EB12CA12CA7
:100900002097B1F08091E80085FD22C08091E80039
:100910008E778093E8006AD401151105A1F0F801E3
:1009200080819181A80EB91EB182A08285E0F82E47
:100930008F2DDF91CF911F910F91FF90DF90CF907E
:10094000BF90AF900895DBD18823D1F2F82EF0CF7D
:10095000F60181916F018093F1002197FFEFAF1AAB
:10096000BF0ACECFAF92BF92CF92DF92FF920F938A
:100970001F93CF93DF936C01EB018A01C0D1F82E56
:10098000811124C00115110539F0F8018081918190
:10099000C81BD90BC80ED91EB12CA12C2097B1F0C1
:1009A0008091E80085FD22C08091E8008B778093DC
:1009B000E8001CD401151105A1F0F8018081918196
:1009C000A80EB91EB182A08285E0F82E8F2DDF918E
:1009D000CF911F910F91FF90DF90CF90BF90AF907C
:1009E00008958DD18823D1F2F82EF0CF8091F100B7
:1009F000F60181936F012197FFEFAF1ABF0ACECFA7
:100A0000FC01809173019091740186179707A0F003
:100A10006115710529F49091E8009E779093E800A4
:100A200090E06115710551F4911108C08091E800C2
:100A300082FF32C080E00895BC01F2CF80916C014A
:100A40008823B1F18530B1F18091E80083FD2EC09B
:100A50008091E80082FDEACF8091E80080FFE1CF3D
:100A60002091F20030E06115710519F02830310550
:100A700058F091E02830310509F090E02091E8002D
:100A80002E772093E800CDCF81918093F1006150C3
:100A900071092F5F3F4FE7CF80916C01882341F0B0
:100AA000853041F08091E80083FFC0CF81E0089558
:100AB00082E0089583E00895FC016115710529F431
:100AC0009091E8009B779093E8006115710531F4EF
:100AD0008091E80080FF1BC080E0089580916C0148
:100AE0008823F9F08530C9F08091E80083FD17C0B4
:100AF0008091E80082FFE9CF8091F200882301F322
:100B00008091F100819361507109B1F7D9CF809143
:100B10006C01882331F08530D9F683E0089581E0B7
:100B2000089582E00895FC01809173019091740111
:100B300086179707A0F06115710529F48091E800E8
:100B40008E778093E80090E06115710551F4911162
:100B500008C08091E80082FF33C080E00895BC01A6
:100B6000F2CF80916C018823B9F18530B9F1809181
:100B7000E80083FD2FC08091E80082FDEACF8091DC
:100B8000E80080FFE1CF2091F20030E061157105AF
:100B900019F02830310558F091E02830310509F07E
:100BA00090E08091E8008E778093E800CDCF84912B
:100BB0008093F1003196615071092F5F3F4FE6CF6E
:100BC00080916C01882341F0853041F08091E800EC
:100BD00083FFBFCF81E0089582E0089583E0089508
:100BE000982F953028F08F708093E90081E0089568
:100BF0009093E900242F762F50E0981731F07091F0
:100C0000EC002091ED005091F00021FD02C09F5FAB
:100C1000E8CF3091EB003E7F3093EB003091ED0058
:100C20003D7F3093ED003091EB0031603093EB006D
:100C30007093EC002093ED005093F0002091EE00B3
:100C400027FDE5CF80E008950F931F93CF93DF93A7
:100C5000062FEC0110E0101302C081E00FC02881C4
:100C6000211103C01F5F2596F6CF9C81A981BA810F
:100C70006B81822F8F70853030F080E0DF91CF91D3
:100C80001F910F91089542E0923008F046E0E8E0AD
:100C9000F0E090E0EA17FB0778F09295907F492BFF
:100CA0006295660F660F607C221F2227221F622B2F
:100CB00097DF8111D7CFE1CF9F5FEE0FFF1FEACF04
:100CC00080916D0187FF13C08091E80082FF06C00C
:100CD0008091E8008B778093E80004C080916C01DC
:100CE0008111F2CF089580916C018823D9F380910E
:100CF000E80080FFF8CF8091E8008E77ECCF20915C
:100D0000E4003091E50085E69091EC0090FF06C08C
:100D10009091E80090FF06C080E008959091E8006F
:100D200092FDFACF90916C01992391F0953091F05A
:100D30009091EB0095FD10C04091E4005091E500CA
:100D40002417350709F381509A01F1F684E00895DC
:100D500082E0089583E0089581E0089541D043D072
:100D60008091D8008F778093D8008091D8008068D8
:100D70008093D8008091D8008F7D8093D80084E044
:100D800089BD86E089BD09B400FEFDCF10926C01DB
:100D90001092680110926A011092690142E060E0CD
:100DA00080E01EDF8091E1008E7F8093E1008091E2
:100DB000E20081608093E2008091E200886080938D
:100DC000E2008091E0008E7F8093E0000895E3E6EA
:100DD000F0E080818E7F808381E080936B01BECFC5
:100DE0001092E20008951092E10008951F920F9270
:100DF0000FB60F9211242F933F934F935F936F93EE
:100E00007F938F939F93AF93BF93EF93FF938091C3
:100E1000E10082FF0AC08091E20082FF06C080915B
:100E2000E1008B7F8093E10087DC8091E10080FF0F
:100E300017C08091E20080FF13C08091E2008E7F96
:100E40008093E2008091E20080618093E2008091D3
:100E5000D80080628093D80019BC10926C0140DBEE
:100E60008091E10084FF27C08091E20084FF23C0CD
:100E700084E089BD86E089BD09B400FEFDCF809184
:100E8000D8008F7D8093D8008091E1008F7E809381
:100E9000E1008091E2008F7E8093E2008091E20089
:100EA00081608093E200809168018823D9F184E019
:100EB00080936C0114DB8091E10083FF22C080915C
:100EC000E20083FF1EC08091E100877F8093E100F4
:100ED00082E080936C01109268018091E1008E7F26
:100EE0008093E1008091E2008E7F8093E200809108
:100EF000E20080618093E20042E060E080E070DE2A
:100F000074D1FF91EF91BF91AF919F918F917F919C
:100F10006F915F914F913F912F910F900FBE0F9066
:100F20001F9018958091E30087FD02C081E0C0CF3B
:100F300083E0BECF1F93CF93DF93CDB7DEB7AA97E1
:100F40000FB6F894DEBF0FBECDBFEDE6F1E08091A5
:100F5000F100819321E0E537F207C9F7D7DB8091F3
:100F6000E80083FF10C080916D0190916E01953073
:100F700009F4D8C000F5913009F48BC008F461C0C1
:100F8000933009F486C08091E80083FF0AC0809105
:100F9000E800877F8093E8008091EB008062809377
:100FA000EB00AA960FB6F894DEBF0FBECDBFDF915F
:100FB000CF911F910895983009F4ECC0993009F44D
:100FC000F6C0963001F780588230E8F680916F01C4
:100FD000909170018C3D23E0920709F0C6C083E038
:100FE0008A838AE289834FB7F894DE01139620E062
:100FF0003EE051E2E32FF0E050935700E49120FFF0
:1010000003C0E295EF703F5FEF708E2F90E0EA3003
:1010100008F4A9C0C7968D939D932F5F243151F793
:101020004FBF8091E800877F8093E8006AE270E01C
:10103000CE010196E5DC8091E8008B778093E80093
:10104000A2CF803899F0823809F09DCF809171014C
:101050008F70853008F097CF8093E9008091EB0086
:1010600085FB882780F91092E90006C0809169010C
:1010700090916A01911182609091E800977F90931E
:10108000E8008093F1001092F1008091E8008E77E3
:1010900032C0282F2D7F09F076CF8823E9F08230E7
:1010A00009F071CF80916F01811120C08091710191
:1010B0008F702FEF280F243008F065CF8093E90060
:1010C0002091EB0020FF12C09330C9F48091EB0017
:1010D00080628093EB000AC080916F01813009F03B
:1010E00052CF933009F080E080936A011092E900BA
:1010F0008091E800877F8093E800E2DD44CF909103
:10110000EB0090619093EB0021E030E001C0220FF2
:101110008A95EAF72093EA001092EA008091EB00AA
:101120008860D7CF81112FCF10916F011F778091E9
:10113000E3008078812B8093E3008091E800877F33
:101140008093E800BDDD8091E80080FFFCCF8091B6
:10115000E30080688093E30083E0111101C082E026
:1011600080936C0110CFC09656CF60917101709141
:101170007201AE014F5F5F4F4ED9BC01892B09F45C
:1011800002CF9091E800977F9093E80089819A813F
:10119000CADC51CF803809F0F6CE8091E800877F15
:1011A0008093E800809168018093F1006ECF8111F7
:1011B000EACE90916F01923008F0E5CE8091E80080
:1011C000877F8093E800909368017ADD80916801C1
:1011D000882329F084E080936C0183D9D4CE809158
:1011E000E30087FDF7CF81E0F6CF0895CF9380919C
:1011F0006C01882391F0C091E900CF708091EC00E0
:1012000080FD0DC080E0C82B1092E9008091E800BD
:1012100083FD90DECF70C093E900CF91089580E800
:06122000F2CFF894FFCFAD
:10122600920074007400B400A000A0000F01C60074
:10123600C600450133012101010000000000000045
:1012460000000000000000FFFF1200290029000234
:0A12560010000301811000030100E5
:00000001FF
